:020000004D2889
:080008004D2863308C000C2030
:100010008D0B052800000800000000000000000013
:100020000000000000008C0B0C2800000800861463
:100030000C200C200C2086100C200C200C20861488
:100040000C200C2086100C200C2086140C2086100E
:100050000C2008308F001720101C33204020900CFB
:100060008F0B2C2808003C308E00861432308D0017
:100070000520861032308D0005208E0B35282F206C
:100080002D308E00861496308D0005208610963017
:100090008D0005208E0B42282F2083160030810012
:1000A00000308B008316F3308500F1308600811715
:1000B00083120301850086008515861006118611BE
:1000C0000230910006158615051D6B20861D6B20DC
:1000D000900A6428602804309200900D920B6D28DD
:0600E000910B29206028AD
:00000001FF
